:1020000092431A020013FFFFFFFFFFFFFFFFFFFFD6
:10201000FFFFFFFFFFFFFFFFFFFFFFFFFFFFFFFFD0
:10202000A107FFFFFFFFFFFFFFFFFFFFFFFFFFFF16
:102080007665722E20352E30202800417072203265
:1020900033203230313500200031303A31323A3499
:1020A00032002900FFFFFFFFFFFFFFFFFFFFFFFFE1
:1020B000FFFFFFFFFFFFFFFFFFFFFFFFFFFFFFFF30
:1020C000FFFFFFFFFFFFFFFFFFFFFFFFFFFFFFFF20
:1020D000FFFFFFFFFFFFFFFFFFFFFFFFFFFFFFFF10
:1020E000FFFFFFFFFFFFFFFFFFFFFFFFFFFFFFFF00
:1020F000FFFFFFFFFFFFFFFFFFFFFFFFFFFFFFFFF0
:1021000092531602925302028263040292B32E0289
:102110001228B2400C5A2001C29334001534B290F8
:10212000F50140011128C243580092C32E02B1C0EC
:10213000D0000000001392532802B29064002802DD
:102140000334B2400C5A20010013FFFFFFFFFFFFD2
:10215000FFFFFFFFFFFFFFFFFFFFFFFFFFFFFFFF8F
:10216000FFFFFFFFFFFFFFFFFFFFFFFFFFFFFFFF7F
:10217000FFFFFFFFFFFFFFFFFFFFFFFFFFFFFFFF6F
:10218000FFFFFFFFFFFFFFFFFFFFFFFFFFFFFFFF5F
:10219000FFFFFFFFFFFFFFFFFFFFFFFFFFFFFFFF4F
:1021A000FFFFFFFFFFFFFFFFFFFFFFFFFFFFFFFF3F
:1021B000FFFFFFFFFFFFFFFFFFFFFFFFFFFFFFFF2F
:1021C000FFFFFFFFFFFFFFFFFFFFFFFFFFFFFFFF1F
:1021D000FFFFFFFFFFFFFFFFFFFFFFFFFFFFFFFF0F
:1021E000FFFFFFFFFFFFFFFFFFFFFFFFFFFFFFFFFF
:1021F000FFFFFFFFFFFFFFFFFFFFFFFFFFFFFFFFEF
:102200003140000A3C4000023D403605B012847A5D
:10221000B0124638B01266790A120B120F4CF2D087
:1022200040000400F240B2007100F240160070005D
:10223000E2427400C2437500C2437300F2D00E0044
:102240001B00D2D31A00D2D31900D2C31900F24016
:10225000C0007700F2B040000200FC2B5A4276002A
:10226000D2D319007D40E0007C400F00B012F2276D
:102270000D12C14F00003D417DD080007C402A00FE
:10228000B012F2277D4024007C402900B012F227D2
:102290006D427C402800B012F2274D437C402B0059
:1022A000B012F2277B4020004F43063C4D434C4B7D
:1022B000B012F2275B535F537F92F82B4B434F438F
:1022C000063C4D434C4BB012F2275B535F537F905B
:1022D0000C00F72B7B4010004F43063C4D434C4B0A
:1022E000B012F2275B535F537F900C00F72B7B40BB
:1022F00030004A430B3C4D434C4BB012F2275B532A
:102300005F537F900E00F72B6B535A537A90030064
:10231000022C4F43F63FE293B9066A207D40C40089
:102320007C405100B012F2277D407E007C402000AE
:10233000B012F2277D427C402100B012F2277D408E
:102340007F007C402200B012F2277D4044004C43C5
:10235000B012F2277D425C43B012F2275D42B8060C
:102360006C43B012F2275D436C42B012F2277D42FB
:102370007C400500B012F2277D4080007C400600C2
:10238000B012F2277D437C402400B012F2277D4238
:102390007C402500B012F2274D437C402600B0124D
:1023A000F2276D427C42B012F2277D427C40090048
:1023B000B012F2276D427C401000B012F2277D422D
:1023C0007C401100B012F2276D427C401400B01224
:1023D000F2277D427C401500B012F2276D427C400E
:1023E0001800B012F2277D427C401900B012F2278B
:1023F000F292B90694207D40C8007C405100B01292
:10240000F2277A4070001F429C051FD29E050F9351
:1024100001206AD28293A20501206AD34D4A7C40F2
:102420002000B012F2277D427C402100B012F2273A
:102430007D407F007C402200B012F2277D404000AA
:102440004C43B012F2277D425C43B012F2275D424A
:10245000B8066C43B012F2274D436C42B012F2271B
:102460007D427C400500B012F2274D437C400600BF
:10247000B012F2277D437C402400B012F2277D4247
:102480007C402500B012F2277D437C402600B0122C
:10249000F2277D437C402700B012F2276D437C4237
:1024A000B012F2277D427C400900B012F2275D4253
:1024B000B8067C400A00B012F2275D42B8067C40A4
:1024C0000B00B012F2276D437C401000B012F227CF
:1024D0007D427C401100B012F2275D42B8067C407C
:1024E0001200B012F2275D42B8067C401300B01211
:1024F000F2276D437C401400B012F2277D427C40ED
:102500001500B012F2275D42B8067C401800B012E8
:10251000F2275D42B8067C401900B012F227F29013
:102520000A00B906F3207D40C2007C405100B01281
:10253000F2277D407E007C402000B012F2277D42D1
:102540007C402100B012F2277D407F007C402200B9
:10255000B012F2277D4042004C43B012F2277D4278
:102560005C43B012F2275D42B8066C43B012F2270A
:102570005D436C42B012F2277D427C400500B012F0
:10258000F2277D4080007C400600B012F227B29016
:102590000500940572247D437C402400B012F2278C
:1025A0007D427C402500B012F2277D437C4026000E
:1025B000B012F2277D437C402700B012F2276D4312
:1025C0007C42B012F2277D427C400900B012F22713
:1025D0005D42B8067C400A00B012F2275D42B806A0
:1025E0007C400B00B012F2276D437C401000B0120B
:1025F000F2277D427C401100B012F2275D42B806FE
:102600007C401200B012F2275D42B8067C401300F5
:10261000B012F2276D437C401400B012F2277D42C5
:102620007C401500B012F2275D42B8067C401600CF
:10263000B012F2275D42B8067C401700B012F227B4
:102640006D437C401800B012F2277D427C40190097
:10265000B012F2275D42B8067C401A00B012F22791
:102660005D42B8067C401B00B012F2277D400A0094
:102670007C400C00B012F227493C7D437C40240092
:10268000B012F2277D40EF007C402500B012F22707
:102690004D437C402600B012F2274D437C4027007A
:1026A000B012F2277D4044007C42B012F2277D40F8
:1026B00028007C400900B012F2277D4044007C4095
:1026C0001000B012F2277D4088007C401100B0124B
:1026D000F2277D4042007C401400B012F2277D4278
:1026E0007C401500B012F2277D4044007C40180069
:1026F000B012F2277D4028007C401900B012F2276A
:102700007D400C007C400C00B012F2277D427C40E2
:102710000500B012F2277D4006007C400F00B01289
:10272000F2277D4003007C402B00B012F2274D437E
:102730007C406000B012F2274D437C407000B01224
:10274000F2275D437C404100B012F2277D427C407D
:102750004200B012F2274D437C404300B012F227F2
:102760005D437C404400B012F2277D4006007C406F
:102770004500B012F2277D427C405200B012F22791
:102780005D42B8067C405300B012F2277D4019002C
:102790007C405400B012F2274D437C405500B012EB
:1027A000F2273B413A4130417D4020007C400F0000
:1027B0003040F227D2C31900F24003007700F2B094
:1027C00040000200FC2B5E427600C24C7700F2B063
:1027D00040000200FC2B5E427600C2437700F2B05C
:1027E00040000200FC2B5E427600D2D319004C4E12
:1027F0003041D2C31900E2437700C2930200FD3793
:10280000C24C7700C2930200FD37C24D7700D2B3AD
:102810007100FD2B5E427600D2D319003041D2C345
:102820001900F24005007700C2930200FD37C24C48
:102830007700C2930200FD37C24E7700C2930200B8
:10284000FD37C24D7700D2B37100FD2B5E4276009A
:10285000D2D319003041D2C31900F24003007700EF
:10286000F2B040000200FC2B5E4276007E40600029
:10287000C24E7700F2B040000200FC2B5E427600B0
:10288000C2437700F2B040000200FC2BD242760037
:102890008E06C2437700F2B040000200FC2BD24209
:1028A00076008F06C2437700F2B040000200FC2B96
:1028B000D24276009006C2437700F2B04000020098
:1028C000FC2BD24276009106C2437700F2B0400062
:1028D0000200FC2BD24276009206C2437700F2B08F
:1028E00040000200FC2BD242760093065E42930623
:1028F0007EF00F004C4E4E935A24C2437700F2B044
:1029000040000200FC2BD242760094065E934F24D6
:10291000C2437700F2B040000200FC2BD2427600A6
:1029200095066E934424C2437700F2B04000020043
:10293000FC2BD242760096067E9003003824C243D8
:102940007700F2B040000200FC2BD24276009706DE
:102950006E922D24C2437700F2B040000200FC2B9F
:10296000D242760098067E9005002124C24377006B
:10297000F2B040000200FC2BD242760099067E9015
:1029800006001524C2437700F2B040000200FC2B81
:10299000D24276009A067E9007000924C24377004F
:1029A000F2B040000200FC2BD24276009B06D2D34C
:1029B00019003041D2C31900F24003007700F2B091
:1029C00040000200FC2B5E4276007E407000C24E4A
:1029D0007700F2B040000200FC2B5E427600C2435A
:1029E0007700F2B040000200FC2BD24276009C0639
:1029F000C2437700F2B040000200FC2BD2427600C6
:102A00009D06C2437700F2B040000200FC2BD24288
:102A100076009E06C2437700F2B040000200FC2B15
:102A2000D24276009F06C2437700F2B04000020017
:102A3000FC2BD2427600A006C2437700F2B04000E1
:102A40000200FC2BD2427600A1065E42A1067EF077
:102A50000F004C4E4E935A24C2437700F2B0400010
:102A60000200FC2BD2427600A2065E934F24C243A2
:102A70007700F2B040000200FC2BD2427600A306A1
:102A80006E934424C2437700F2B040000200FC2B56
:102A9000D2427600A4067E9003003824C243770019
:102AA000F2B040000200FC2BD2427600A5066E92E6
:102AB0002D24C2437700F2B040000200FC2BD2422A
:102AC0007600A6067E9005002124C2437700F2B06E
:102AD00040000200FC2BD2427600A7067E90060042
:102AE0001524C2437700F2B040000200FC2BD24212
:102AF0007600A8067E9007000924C2437700F2B052
:102B000040000200FC2BD2427600A906D2D3190065
:102B100030417E434D437C402C0030401E28D2C3C0
:102B20001900E2437700C2930200FD37F240310002
:102B300077003D4081065F4285067FF00F007F50A1
:102B400005004E43073CC2930200FD37E24D77007B
:102B50001D535E534E9FF72BD2B37100FD2B5E4287
:102B60007600D2D319004E43D2C31900F24081003F
:102B70007700F2B040000200FC2B5E427600D2D318
:102B800019003041D2C319004E43F2408100770052
:102B9000F2B040000200FC2B5E427600D2D3190056
:102BA00030410A125A42AF064A4A3AF00F003A50F0
:102BB00006001F430B3C5D4FAA060C12C14F0000DC
:102BC0003C417C504000B012F2271F530F9AF33B58
:102BD000D2C31900F24082007700F2B04000020038
:102BE000FC2B5F4276004F4FD2D319003A4130415F
:102BF000FC902D0000002D20DC9304002A20FC9086
:102C00000600020026205E4C06004E4E3E5038FF65
:102C10000E5E5F4C09004F4F1FE31FF30E5FCC9316
:102C200009000B3482934E041F20B24005004E046D
:102C300082435604824E50043041B29005004E0447
:102C40001320829E50041020A2D34E0482435204CB
:102C50003041FC90670000000724FC9064000000F5
:102C60000320B24000015A0430410A120B1208122C
:102C700082935A0602243040E43192B36E0626282D
:102C80009243740682436E0682437C068243780632
:102C900082437A061F4270060F5F824F7606B2406B
:102CA00000025A04F2406800C406E242C506F2403F
:102CB0000B00C606C243C706C243C806C243C906C4
:102CC0003C400600B0122C353040E431829374064B
:102CD00002203040E431A2B36E061628A2C36E066D
:102CE000F2406800C406E242C506F2408300C60610
:102CF000C243C706C243C806C243C9063C400600D9
:102D0000B0122C353040E431A2B26E061628824350
:102D10006E06F2406800C406E242C506F240230097
:102D2000C606C243C706C243C806C243C9063C40E2
:102D30000600B0122C353040E431929276067C06C3
:102D40000528B2400A0072063040E4313A400600DD
:102D5000B29000025A04232082435A04FA404600EB
:102D6000C4061A53DA43C4061A53EA42C4061A5375
:102D7000CA43C4061A53DA43C4061A53CA43C406E4
:102D80001A53CA43C4061A53CA43C4061A53CA4341
:102D9000C4061A53EA43C4061A533040A631A2B2FD
:102DA0004E043928A29356043620FA402D00C4065A
:102DB0001A53DA43C4061A53FA400700C4061A53DA
:102DC000CA43C4061A53DA43C4061A53CA43C40694
:102DD0001A531E42500412C30E107E50C800CA4E31
:102DE000C4061A53CA43C4061A53CA43C4061A5324
:102DF0005E4250045EE35EF37E508000CA4EC4061D
:102E00001A53B24003005604B2D000806806B240A4
:102E100032005204C83DA2B24E043528B2900500DB
:102E200056043120FA402D00C4061A53DA43C40672
:102E30001A53FA400700C4061A53CA43C4061A5369
:102E4000DA43C4061A53CA43C4061A531E42500436
:102E500012C30E107E50C800CA4EC4061A53CA438D
:102E6000C4061A53CA43C4061A535E4250045EE3B2
:102E70005EF3CA4EC4061A53B24006005604B2D0DE
:102E800000406806903DA2B24E043828B290060079
:102E900056043420FA402D00C4061A53DA43C406FF
:102EA0001A53FA400A00C4061A53CA43C4061A53F6
:102EB000DA43C4061A53CA43C4061A531E425004C6
:102EC00012C30E107E50C800CA4EC4061A53CA431D
:102ED000C4061A53CA43C4061A535E4250045EE342
:102EE0005EF3CA4EC4061A538243560482434E040C
:102EF00082435804B240FF005004553DB290000197
:102F00005A042520B24006035A04FA406400C4065D
:102F10001A53DA43C4061A53FA400700C4061A5378
:102F2000CA43C4061A53DA43C4061A53CA43C40632
:102F30001A53CA43C4061A53CA43C4061A53CA438F
:102F4000C4061A53FA401400C4061A532C3DB2901A
:102F500000045A04242082435A04FA406400C40640
:102F60001A53DA43C4061A53FA400A00C4061A5325
:102F7000CA43C4061A53DA43C4061A53CA43C406E2
:102F80001A53CA43C4061A53CA43C4061A53CA433F
:102F9000C4061A53FA401400C4061A53043D1F42D3
:102FA00048043FF01F001F924A044724DA43C40636
:102FB0001A53DA43C4061A53FA400300C4061A53DC
:102FC000CA43C4061A53DA43C4061A53CA43C40692
:102FD0001A531F424A041F533FF01F000F5F0F5F39
:102FE0000F5F5E4F48037EF07F005E535F429605A1
:102FF0004F5F4F5F4E8FCA4EC4061A53CA43C40672
:103000001A53CA43C4061A530F4A0A4F1A531B4293
:103010004A041B533BF01F000B5B0B5B0B5BCB931A
:10302000480302385E43013C4E43CF4EC4069253E0
:103030004A04B2F01F004A04B63CA2B25A044A281D
:10304000A2C25A041F425A043FF000033F900003FB
:1030500041203F4020001B4296050B5B0B5B0F8B12
:103060000F933824DA43C4061A530E12C14F0000DE
:103070003E417E508000CA4EC4061A53FA401400E6
:10308000C4061A53CA43C4061A53DA43C4061A5371
:10309000CA43C4061A53DA43C4061A53CA43C406C1
:1030A0001A53CA43C4061A530B43113C1C4244032F
:1030B0001D4246035E4296054E5E4E5E4E5BB0126A
:1030C0004A7A5CF35CE3CA4CC4061A531B530B9F49
:1030D000ED3B693CF2B003005A046524B2F0FCFFFA
:1030E0005A041F4296050F5F0F5F0F935C24FA404E
:1030F0000900C4061A530E12C14F00003E417E5013
:103100008000CA4EC4061A531B425A043BF0000307
:103110003B9000030820FA401400C4061A53B24042
:1031200000045A04043CFA400300C4061A53CA437C
:10313000C4061A53DA43C4061A53CA43C4061A53C0
:10314000FA406400C4061A53CA43C4061A53CA4359
:10315000C4061A53B24076021E020B4A3B50C40604
:10316000824B1C020B431D3C1E421E021D421C02D0
:10317000ED4E000092531E0292531C021E421E028C
:103180001D421C02ED4E000092531E0292531C027F
:103190001E421C02CE43000092531C023A50030010
:1031A0001B530B9FE13B3A9007001C38F24068002C
:1031B000C4060E12C14A00003E417E50FE00C24EBF
:1031C000C506D2427C06C606D2427D06C706D2425A
:1031D0007806C806D2427906C906A2537C060C4A74
:1031E000B0122C35304076790F120E128293A8055A
:1031F000162092925A065C0608341F425C06D24F93
:10320000C4067F0092535C06523CF2C020000100CD
:10321000D2C329008243660682435A06483CB290D4
:1032200000105C060438B24000205C06403CB290BE
:1032300001045C060620F24068007F0092535C06A1
:10324000363CB29002045C060424B29003045C068F
:1032500008205E425A067E53C24E7F0092535C069F
:10326000263CB29004045C060620F24068007F0011
:1032700082435C061C3CB29001055C060620F240CD
:1032800010007F0082435C06123C92925A065C0654
:1032900008341F425C06D24FC4067F0092535C067E
:1032A000063CF24016007F00B24000105C063E4132
:1032B0003F4100130D120C120F120E12D2B37A00FE
:1032C0000628D2427E001407F2427A00073DD2421D
:1032D0007E0014078293A8057C20B29020006A0625
:1032E000052C1F426A06DF421407150792536A062F
:1032F00092936A060720F29068001407EF24824335
:103300006A06EC3CA2936A0607205F4214074F4FFF
:103310002F53824F6C06E23C92926C066A06DE28BE
:1033200082432602B29006006A062C2082436A0677
:103330005E4217075E8313247E80060007247E808A
:103340000C000A247E8030000424C83C92436E06A0
:10335000C53CA2D36E06C23CA2D26E06BF3C8243DD
:1033600072065E4219074E4E5F421A074F4F3FF0FA
:10337000FF008F100E5F1F4270060F5F0E5F824EC0
:103380007606AC3C5E4219074E4E5F421A074F4F1D
:103390003FF0FF008F100E5F1F4270060F5F0E5F41
:1033A000824E76065E4217074E4E5F4218074F4F19
:1033B0003FF0FF008F100E5F824E7806A253780612
:1033C000B2D26E063C401B07B012F02B82436A0655
:1033D000853C82935E068220B29000025C06122039
:1033E000F29068001407032092535C06773CF29039
:1033F00010001407732082437E0682435C06A243BA
:103400005A066C3CB29001025C0610205F42140721
:103410004F4F824F5A06B29050005A060438B240BD
:1034200000025C065B3C92535C06583CB290020280
:103430005C060D205F4214074F4F829F5A060424FA
:10344000B24000025C064A3C92535C06473CB29094
:1034500003025C060D20F290680014070424B240B9
:1034600000025C063B3C82435C0682437E06363C9F
:1034700092925A065C060F341F425C06DF42140724
:10348000C4061F425C065F4FC4064F4F825F7E0634
:1034900092535C06233C92925A065C060D205E42D3
:1034A0007E067EF35E9214070424B24000025C069E
:1034B000153C92535C06123CB29000015C060E343F
:1034C000F290160014070424B24000025C06063C89
:1034D000B24005005E06F2C0100001003E413F41CF
:1034E0003C413D41001382437E060E43063C5F4E45
:1034F000C4064F4F825F7E061E530E9CF82BDE42A1
:103500007E06C4061C533C9003000420B240010513
:103510005C06033CB24001045C0692435E068243B3
:10352000640682436206824C5A063041824C5A0637
:1035300082435C06D2D32900F2D020000300F2D0EF
:1035400020000100304182435E0682436206B240A1
:1035500000025C06F2D0100001008293A805082446
:1035600082435A06F2C020000100F2C0200003008E
:103570003041F2D030000500F2D010007800F2D0D7
:10358000C0001B00F2D0200079001F42AA053FF0C6
:103590000F000E4F0F5F0F5ED24FE47A7C001F4288
:1035A000AA053FF00F000E4F0F5F0F5ED24FE57A76
:1035B0007D001F42AA053FF00F000E4F0F5F0F5E08
:1035C000D24FE67A7B008293A8050424F240D00013
:1035D0007800033CF24010007800F2427A001F426B
:1035E000AA058F103FF0FF00824F6006B2400C002A
:1035F0007006B012463582436806824374060F4354
:10360000824F6406824F6606824F62061F42700137
:103610003F500A003FF0FF03824F760130410A120B
:103620004F4CB2900600820596383C4003000D4393
:103630004E4F7EF01E00B0121E7A82BC9C05032005
:1036400082BD9E053C244A4F3AF01E003AD020002D
:103650001C4236021D4238024E4F7EF01E00B01250
:103660004A7A3CF003005FB3782C2CB302283AD09E
:1036700040004F9310343AD080001CB3092C2CB377
:103680001A284F4F3FF01F000F5F8F430205633C26
:103690002CB3112C603C1CB30E282CB30C2C4E4FB9
:1036A0003EF01F000E5E4F4F3FF01F000F5F9F4E1A
:1036B00042050205503C0F12C14A00003F4192539F
:1036C000BA031C42BA033CF01F001C92BC03072043
:1036D0001E42BC031E533EF01F00824EBC034F4FE0
:1036E0000E4C0E5E0E5E0E5E8E4FBA020F4C0F5FDA
:1036F0000F5F0F5F9F420202BC029F420402BE02A4
:103700001F427001021232C20343824F3001B240A5
:10371000E80338011E423A011F423C0132413E504B
:1037200000020F638E108F104EEF0EEF3FF0FF0080
:10373000824E0602824F080212C3121008021210B3
:10374000060212110802121006020C5C0C5C0C5CE2
:103750009C420602C0023A4130411CB302283AD0D2
:1037600080004F9310343AD040002CB3092C1CB386
:10377000A22B4F4F3FF01F000F5F8F430205EB3F1F
:103780001CB3992FE83F2CB30E281CB3942F4E4F37
:103790003EF01F000E5E4F4F3FF01F000F5F9F4E29
:1037A00042050205D83F1CB3862BD53F92534804EF
:1037B0001E4248043EF01F001E924A0407201F428A
:1037C0004A041F533FF01F00824F4A044C4C0F4ED7
:1037D0000F5F0F5F0F5F8F4C48030F4E0F5F0F5F40
:1037E0000F5F9F4202024A039F4204024C031F42A2
:1037F0007001021232C20343824F3001B240E8032B
:1038000038011C423A011D423C0132413C50000249
:103810000D638C108D104CED0CED3DF0FF00824CD3
:103820000602824D080212C312100802121006028C
:1038300012110802121006020E5E0E5E0E5E9E420D
:1038400006024E0330410A120B1208128243000294
:10385000C243BE0682432E0282431A0282432802DA
:10386000C243BF06F2F040003600F2B04000340020
:103870000328B2D000012E02E2B234000328B2D0F5
:1038800000052E02F2C020001900F2D020001A001C
:10389000B240805A2001C243000032C20343384084
:1038A0003C000A3C5B4280205B428B205B429920BB
:1038B0005B4297205B42A2200F48084F38530F937A
:1038C000F1233F4000211F92ECFF0F203F40E831E1
:1038D0001F92E4FF0A203F40B4321F92E6FF05200A
:1038E0003F4000201F92FCFF7B24F2402400570041
:1038F000E2C302000843023C1A5318533890FF00F9
:10390000FB2BE2B30200F42FF2D25800F240880001
:103910005800B24051A52A01B24002A52801B24088
:1039200000A52C018243E0FFB24000A52801B2406F
:1039300010A52C01B24040A52801B24000A52C01E1
:10394000B2400021ECFFB24000A52801B24010A512
:103950002C01B24040A52801B24000A52C01B24084
:10396000E831E4FFB24000A52801B24010A52C01C7
:10397000B24040A52801B24000A52C01B240B432AB
:10398000E6FFB24000A52801B24010A52C01B240CC
:1039900040A52801B24000A52C01B2400020FCFF48
:1039A000B24000A52801B24010A52C01B24040A5AC
:1039B0002801B24000A52C01B2400022FEFFB24017
:1039C00000A52801B24010A52C018243600182436A
:1039D000800132D282430002B2400B5A2001FF3FE5
:1039E000F240A4005700B240C0016001B240FF03A2
:1039F0007201B2D010006001B2401000620132D2F8
:103A0000B2400C5A200182432002663C0B12C14A8C
:103A100000003B4112C34B104B114B114B4B3BF081
:103A200003005F429F064F4F0F5F0F5F0B5F5C43CA
:103A30000E12C14A00003E417EF00700B012127A19
:103A4000CBCC5E02C2933400023430408C3FB012C3
:103A5000A827B2900B0020020238B0127E75C24334
:103A60002600C2432200C2432E00C2432A00C243A2
:103A70001B00C2431A00C2431F00C2431E00C243C0
:103A80003300C2433200C2433700C2433600F24023
:103A9000C0005800C2431B00C2431A00F240A000FD
:103AA0005700C243000092D32E02F240200037009C
:103AB000B2401007A001B2400402A201F24085000A
:103AC000800082434001A2D3A00192D3A00132D052
:103AD000D000F240A4005700F24020003700B2406E
:103AE0001007A001B2400002A201F2408500800050
:103AF000023CB0121479A2D3A00192D3A00192B3D8
:103B0000A201FD2FA2D3A00192D3A00192B3A201E2
:103B1000FD2FB290F4014001042C82932002E9278A
:103B20009E3F8243A001C2433700F2402400570069
:103B3000E2C302000843023C1A5318533890FF00B6
:103B4000FB2BE2B30200F42FF2D25800F2408800BF
:103B5000580082432002B0124A7682932202032048
:103B6000D243BD06043CC243BD0692439205B2B0A7
:103B700000012E020628F24040003600F2C040004C
:103B80003500B2B000042E020428E2D23600E2C2B0
:103B90003500F292B9062920B2B000012E02202889
:103BA000B2D000022E02C2432100C2432900F2C05B
:103BB00010001900C2431D00C2433100F24322002D
:103BC000F2407F002A00F2D010001A00F2431E00DB
:103BD000F2433200D242227B1D00B0127235053C06
:103BE000F2432200D242027B2100F2900A00B90681
:103BF0001420C2432100C2432900C2431D00C24316
:103C00003100F2C010001900F2D010001A00F2C00A
:103C100020001900F2D020001A000C43B012182224
:103C2000F24038003700F2900A00B9061020B24086
:103C3000F007A001B240B202A201F24013008000DE
:103C4000F24015008100F2409A008200173CB24019
:103C5000F003A001B2401202A201B2B000042E0291
:103C60000728F24023008000F240A4008100063CB7
:103C7000F24013008000F24094008100D243BA0663
:103C8000C243BC06D243BB06F2428206C24381064F
:103C9000F24010008406C2438506F292B9066A20FB
:103CA000B290090096050238B2429605F240C8006B
:103CB0008106C243C00682433603824338038243EF
:103CC0003A03C243C206C243C10682434C04824344
:103CD000560482434E0482435804B240FF0050040D
:103CE000824352041C4202021D4204023E40100E56
:103CF0000F43B0129A790A4E1B4294050C4A1E4299
:103D00009405B01282790B8E0E4B0F431E520202A5
:103D10001F620402824E0A02824F0C021B429A0565
:103D20000C4A1E429A05B01282790B8E0E4B0F433D
:103D30001E5202021F620402824E0E02824F1002C5
:103D4000B2B000012E020E285E421C007EF0800000
:103D50005F42C0064F4F3FF01F005EDF227BC24E26
:103D60001D00083C5F42C0064F4F3FF01F00D24F7E
:103D7000027B2100F2900A00B9064720F240C200FF
:103D80008106B290050094052A2082439603F2D062
:103D90002000190082439403C243AA03C243A9032B
:103DA0008243AE038243AC030A43053C0F4A0F5FD4
:103DB0008F433E021A533A92F92B0A43053CCA43F9
:103DC0003A02CA4336021A532A92F92B0A433A900E
:103DD00000011B2CFA4080007E021A53F83F8243F8
:103DE0005602B2900B00940504208243940592433E
:103DF0005602824340028243360282433C0282439F
:103E00003E0292433A02B012122BE293B906872087
:103E1000F240C4008106B2902000BC03042CB29092
:103E20002000BA0304288243BC038243BA039242AF
:103E300036022A02924238022C0208430D3C0B48FB
:103E40000B5B0F480F5F9F4B4205020512C3121018
:103E50002C0212102A021853389020002E2C0F48E2
:103E60000F5F8F93A00505240F480F5FBF93A00538
:103E700013208293A0050B240F480F5FBF93A0056A
:103E800006240F480F5F9F42A005A005053C0F4880
:103E90000F5FBF401400A0050F480F5F1B4FA00528
:103EA0000B5B0F480F5F8F4B420592B32A02C72F5F
:103EB0000F480F5F8F430205C93F8243FE048243D0
:103EC00000051C4202021D4204023E40100E0F4338
:103ED000B0129A790A4E1B4294050C4A1E42940570
:103EE000B01282790B8E0E4B0F431E5202021F62DC
:103EF0000402824E0A02824F0C021B4296050C4AB3
:103F00001E429605B01282790B8E0E4B0F431E5245
:103F100002021F620402824E0E02824F10021C43F4
:103F2000B0128278A2422602B240A00280018243EF
:103F3000820182438601E293B90606201F42900166
:103F40003F50EE02824F9201F2900A00B90606201D
:103F50001F4290013F50DC05824F9201F292B90658
:103F600008201F4290013F50983A824F92018243AD
:103F7000940192D3A001A2D3A0017E434D437C4083
:103F80002C00B0121E28023C82433A0292531202C5
:103F900082631402829316023924824312028243FE
:103FA00014021A42700192B302020328B01214796B
:103FB000023CB0123C79E293B9060620B2900A00A6
:103FC0008205023492538205B2902C0126021034ED
:103FD000C293BD06132492532602B2901500260206
:103FE0000D3892B326020A2C0C43B0121822063C5C
:103FF000B0127E753C400500B0128278B290580233
:10400000200202349253200282431602B2900B0027
:1040100026020C38B290320070010220B0123C79B6
:10402000B290960070010220B0121479C293BD06BE
:10403000022030406869E293B90602243040B05350
:1040400092B3A201082C924240018405924242019F
:10405000860592D3A00192B38201022C3040F84F22
:10406000824382011F4290013F50EE02824F920133
:10407000C293BF062D24C293BC060724B012842B22
:1040800092538A0592532402233CC293BB062024F8
:10409000D242B8068306E293BB060E20F2428206A5
:1040A000C2438106F2438406C2438506F240C4003F
:1040B0008106C243BB060A3CC29381060538C2434F
:1040C000BA06D2428106BC06D2C3BB06B0121E2B72
:1040D000A292200202343040F84F82432802584214
:1040E0002000484818B3202892924205020504286F
:1040F0009242420502052E3C925302059292A0057F
:104100000205282092424205020592B3980505282F
:1041100092533A0282633C02043C7C408000B0121D
:104120001E3692D33602163C829302050320824348
:104130000205103CB25302059292A00502050A2026
:104140008243020592B39805032C4C43B0121E36ED
:1041500092C3360228B3202892924405040504280D
:104160009242440504052E3C925304059292A20506
:1041700004052820924244050405A2B398050528A9
:1041800092533E0282634002043C7C408100B012A4
:104190001E36A2D33602163C8293040503208243C6
:1041A0000405103CB25304059292A20504050A20AE
:1041B00082430405A2B39805032C5C43B0121E365B
:1041C000A2C3360228B2202892924605060504288A
:1041D0009242460506052E3C925306059292A4058E
:1041E00006052820924246050605A2B29805052834
:1041F0009253420282634402043C7C408200B0122B
:104200001E36A2D23602163C829306050320824354
:104210000605103CB25306059292A40506050A2035
:1042200082430605A2B29805032C6C43B0121E36D9
:10423000A2C2360238B22028929248050805042806
:104240009242480508052F3C925308059292A60514
:1042500008052920924248050805B2B298050528AC
:104260009253460282634802043C7C408300B012B1
:104270001E36B2D23602173C8293080503208243D1
:104280000805113CB25308059292A60508050B20BB
:1042900082430805B2B29805042C7C400300B0129A
:1042A0001E36B2C2360238B01000222892924A0559
:1042B0000A05042892424A050A05323C92530A052F
:1042C0009292A8050A052C2092424A050A05B2B02E
:1042D00010009805052892534A0282634C02043C60
:1042E0007C408400B0121E36B2D010003602183C5A
:1042F00082930A05032082430A05123CB2530A0541
:104300009292A8050A050C2082430A05B2B010005B
:104310009805032C6C42B0121E36B2C01000360253
:1043200038B02000222892924C050C0504289242B5
:104330004C050C05333C92530C059292AA050C05D2
:104340002D2092424C050C05B2B02000980505289E
:1043500092534E0282635002043C7C408500B012AE
:104360001E36B2D020003602193C82930C05032081
:1043700082430C05133CB2530C059292AA050C051E
:104380000D2082430C05B2B020009805042C7C401F
:104390000500B0121E36B2C02000360238B0400010
:1043A000222892924E050E05042892424E050E05D3
:1043B000333C92530E059292AC050E052D2092428D
:1043C0004E050E05B2B040009805052892535202E2
:1043D00082635402043C7C408600B0121E36B2D088
:1043E00040003602193C82930E05032082430E05DD
:1043F000133CB2530E059292AC050E050D2082437C
:104400000E05B2B040009805042C7C400600B012A6
:104410001E36B2C0400036024893213492925005B5
:1044200010050428924250051005313C92531005A6
:104430009292AE0510052B20924250051005C293B2
:10444000980505349253560282635802043C7C401E
:104450008700B0121E36B2D080003602183C82931C
:104460001005032082431005123CB25310059292AE
:10447000AE0510050C2082431005C2939805043840
:104480007C400700B0121E36B2C08000360258428F
:104490002800484818B32228929252051205042891
:1044A000924252051205323C925312059292B00587
:1044B00012052C20924252051205B2B00001980557
:1044C000052892535A0282635C02043C7C408800B7
:1044D000B0121E36B2D000013602183C829312058B
:1044E000032082431205123CB25312059292B0058A
:1044F00012050C2082431205B2B000019805032C6E
:104500007C42B0121E36B2C00001360228B3222807
:104510009292540514050428924254051405333C24
:10452000925314059292B20514052D20924254051F
:104530001405B2B000029805052892535E0282630A
:104540006002043C7C408900B0121E36B2D00002EA
:104550003602193C82931405032082431405133C50
:10456000B25314059292B20514050D20824314052E
:10457000B2B000029805042C7C400900B0121E362F
:10458000B2C00002360228B22228929256051605C1
:104590000428924256051605333C92531605929212
:1045A000B40516052D20924256051605B2B000043A
:1045B000980505289253620282636402043C7C40A1
:1045C0008A00B0121E36B2D000043602193C829323
:1045D0001605032082431605133CB253160592922A
:1045E000B40516050D2082431605B2B000049805E7
:1045F000042C7C400A00B0121E36B2C00004360201
:1046000038B222289292580518050428924258057B
:104610001805333C925318059292B60518052D20C3
:10462000924258051805B2B0000898050528925323
:10463000660282636802043C7C408B00B0121E3626
:10464000B2D000083602193C829318050320824339
:104650001805133CB25318059292B60518050D20A3
:1046600082431805B2B000089805042C7C400B006A
:10467000B0121E36B2C00008360238B01000222830
:1046800092925A051A05042892425A051A05333C9B
:1046900092531A059292B8051A052D2092425A0596
:1046A0001A05B2B000109805052892536A02826379
:1046B0006C02043C7C408C00B0121E36B2D000105C
:1046C0003602193C82931A05032082431A05133CD3
:1046D000B2531A059292B8051A050D2082431A05A5
:1046E000B2B000109805042C7C400C00B0121E36AD
:1046F000B2C00010360238B02000222892925C0529
:104700001C05042892425C051C05333C92531C0591
:104710009292BA051C052D2092425C051C05B2B090
:1047200000209805052892536E0282637002043CB3
:104730007C408D00B0121E36B2D000203602193CEB
:1047400082931C05032082431C05133CB2531C05B5
:104750009292BA051C050D2082431C05B2B00020C0
:104760009805042C7C400D00B0121E36B2C000200B
:10477000360238B04000222892925E051E050428B9
:1047800092425E051E05333C92531E059292BC0573
:104790001E052D2092425E051E05B2B00040980510
:1047A00005289253720282637402043C7C408E009E
:1047B000B0121E36B2D000403602193C82931E055C
:1047C000032082431E05133CB2531E059292BC0582
:1047D0001E050D2082431E05B2B000409805042C32
:1047E0007C400E00B0121E36B2C000403602F2B05D
:1047F000100018002128929260052005042892429A
:1048000060052005313C925320059292BE0520059B
:104810002B2092426005200582939805053492531F
:10482000760282637802043C7C408F00B0121E3610
:10483000B2D000803602183C8293200503208243C8
:104840002005123CB25320059292BE0520050C2093
:10485000824320058293980504387C400F00B012F3
:104860001E36B2C000803602584230004848489395
:1048700020349292620522050428924262052205A4
:104880002F3C925322059292C00522052920924284
:104890006205220592B39A05052892537A02826333
:1048A0007C02043C7C409000B0121E3692D3380249
:1048B000173C82932205032082432205113CB25308
:1048C00022059292C00522050B208243220592B355
:1048D0009A05042C7C401000B0121E3692C3380298
:1048E00038B04000202892926405240504289242A2
:1048F000640524052F3C925324059292C205240599
:104900002920924264052405A2B39A0505289253F2
:104910007E0282638002043C7C409100B0121E360D
:10492000A2D33802173C8293240503208243240536
:10493000113CB25324059292C20524050B208243F8
:104940002405A2B39A05042C7C401100B0121E3637
:10495000A2C3380238B020002028929266052605AE
:1049600004289242660526052F3C92532605929212
:10497000C40526052920924266052605A2B29A059D
:1049800005289253820282638402043C7C40920098
:10499000B0121E36A2D23802173C8293260503209D
:1049A00082432605113CB25326059292C405260582
:1049B0000B2082432605A2B29A05042C7C401200EB
:1049C000B0121E36A2C2380238B0100020289292CF
:1049D0006805280504289242680528052F3C925353
:1049E00028059292C60528052920924268052805C7
:1049F000B2B29A0505289253860282638802043C6B
:104A00007C409300B0121E36B2D23802173C82931B
:104A10002805032082432805113CB25328059292B1
:104A2000C60528050B2082432805B2B29A05042C3E
:104A30007C401300B0121E36B2C2380238B22228AF
:104A400092926A052A05042892426A052A05333C97
:104A500092532A059292C8052A052D2092426A0592
:104A60002A05B2B010009A05052892538A02826383
:104A70008C02043C7C409400B0121E36B2D0100070
:104A80003802193C82932A05032082432A05133CED
:104A9000B2532A059292C8052A050D2082432A05A1
:104AA000B2B010009A05042C7C401400B0121E36DF
:104AB000B2C01000380228B2222892926C052C0550
:104AC000042892426C052C05333C92532C0592929B
:104AD000CA052C052D2092426C052C05B2B0200091
:104AE0009A05052892538E0282639002043C7C4012
:104AF0009500B0121E36B2D020003802193C8293C5
:104B00002C05032082432C05133CB2532C059292B2
:104B1000CA052C050D2082432C05B2B020009A0551
:104B2000042C7C401500B0121E36B2C020003802A2
:104B300028B3222892926E052E05042892426E0513
:104B40002E05333C92532E059292CC052E052D2036
:104B500092426E052E05B2B040009A050528925388
:104B6000920282639402043C7C409600B0121E368E
:104B7000B2D040003802193C82932E0503208243B4
:104B80002E05133CB2532E059292CC052E050D2016
:104B900082432E05B2B040009A05042C7C401600DA
:104BA000B0121E36B2C04000380218B321289292CB
:104BB000700530050428924270053005313C92534F
:104BC00030059292CE0530052B20924270053005BB
:104BD000C2939A0505349253960282639802043C6C
:104BE0007C409700B0121E36B2D080003802183CCC
:104BF00082933005032082433005123CB2533005C6
:104C00009292CE0530050C2082433005C2939A055E
:104C100004387C401700B0121E36B2C08000380243
:104C200058421C004848489322349292720532053B
:104C30000428924272053205333C92533205929217
:104C4000D00532052D20924272053205B2B0000126
:104C50009A05052892539A0282639C02043C7C4088
:104C60009800B0121E36B2D000013802193C82936F
:104C70003205032082433205133CB253320592922F
:104C8000D00532050D2082433205B2B000019A05ED
:104C9000042C7C401800B0121E36B2C0000138024D
:104CA00038B04000222892927405340504289242BC
:104CB00074053405333C925334059292D205340581
:104CC0002D20924274053405B2B000029A050528E1
:104CD00092539E028263A002043C7C409900B01271
:104CE0001E36B2D000023802193C829334050320EC
:104CF00082433405133CB25334059292D2053405F5
:104D00000D2082433405B2B000029A05042C7C4089
:104D10001900B0121E36B2C00002380238B02000AE
:104D200022289292760536050428924276053605A9
:104D3000333C925336059292D40536052D2092428B
:104D400076053605B2B000049A0505289253A202F2
:104D50008263A402043C7C409A00B0121E36B2D09A
:104D600000043802193C829336050320824336053D
:104D7000133CB25336059292D40536050D2082437A
:104D80003605B2B000049A05042C7C401A00B0121B
:104D90001E36B2C00004380238B0100022289292A9
:104DA000780538050428924278053805333C92533B
:104DB00038059292D60538052D209242780538059F
:104DC000B2B000089A0505289253A6028263A80291
:104DD000043C7C409B00B0121E36B2D00008380262
:104DE000193C82933805032082433805133CB253A3
:104DF00038059292D60538050D2082433805B2B0A9
:104E000000089A05042C7C401B00B0121E36B2C06C
:104E10000008380238B2222892927A053A0504280E
:104E200092427A053A05333C92533A059292D8055C
:104E30003A052D2092427A053A05B2B000109A0543
:104E400005289253AA028263AC02043C7C409C0079
:104E5000B0121E36B2D000103802193C82933A05C7
:104E6000032082433A05133CB2533A059292D80587
:104E70003A050D2082433A05B2B000109A05042C81
:104E80007C401C00B0121E36B2C00010380228B29E
:104E9000222892927C053C05042892427C053C0520
:104EA000333C92533C059292DA053C052D20924208
:104EB0007C053C05B2B000209A0505289253AE024D
:104EC0008263B002043C7C409D00B0121E36B2D01A
:104ED00000203802193C82933C05032082433C05A4
:104EE000133CB2533C059292DA053C050D208243F7
:104EF0003C05B2B000209A05042C7C401D00B01285
:104F00001E36B2C00020380228B3222892927E05B5
:104F10003E05042892427E053E05333C92533E05F1
:104F20009292DC053E052D2092427E053E05B2B0F0
:104F300000409A0505289253B2028263B402043CF1
:104F40007C409E00B0121E36B2D000403802193CA0
:104F500082933E05032082433E05133CB2533E0537
:104F60009292DC053E050D2082433E05B2B0004022
:104F70009A05042C7C401E00B0121E36B2C00040C0
:104F8000380218B3212892928005400504289242E5
:104F900080054005313C925340059292DE05400564
:104FA0002B2092428005400582939A050534925346
:104FB000B6028263B802043C7C409F00B0121E36E9
:104FC000B2D000803802183C82934005032082430F
:104FD0004005123CB25340059292DE0540050C207C
:104FE0008243400582939A0504387C401F00B0122A
:104FF0001E36B2C0008038021F42BA033FF01F00C5
:105000001F92BC036C24C293BB0602205E43013C8A
:105010004E435F42BA065FF34FBE61249253BC0316
:10502000B2F01F00BC031A42BA033AF0E0FF1A5272
:10503000BC03829ABA03022C3A50E0FFF2404400CB
:1050400081061F42BC030F5F0F5F0F5FD24FBA0292
:105050008406F24285061F42BC030F5F0F5F0F5F9D
:10506000D24FBC0286061F42BC030F5F0F5F0F5F6B
:10507000D24FBD0287061F42BC030F5F0F5F0F5F59
:105080001E4FBE02C24E88061F42BC030F5F0F5F59
:105090000F5F1E4FBC021F4FBE028F104E4F0F43BB
:1050A000C24E89061F42BC030F5F0F5F0F5FD24FD6
:1050B000C0028A061F42BC030F5F0F5F0F5FD24F13
:1050C000C1028B06C24A8C060F4A8F103FF0FF00C8
:1050D000C24F8D06F24088008206D243BB069292F0
:1050E0000C0204021528042092920A0202021028DF
:1050F000829394050D241E4294050F431E52020212
:105100001F620402824E0A02824F0C02D2D3BE06F4
:105110009292100204021528042092920E020202BA
:105120001028829396050D241E4296050F431E52A9
:1051300002021F620402824E0E02824F1002E2D36C
:10514000BE06D2B3BE064528C293BB0602205E430C
:10515000013C4E435F42BA065FF34FBE3A24B2931E
:1051600098050320B2939A0532241E4236021F424C
:1051700038021ED298051FD29A05824E2A02824F0B
:105180002C02F24044008106C2438406F24006002D
:105190008506D2422A028606D2422B0287061E428A
:1051A0002C02C24E88061E422A021F422C028F1079
:1051B0004E4F0F43C24E8906D242BA038A06D242EC
:1051C000BB038B06F24028008206D243BB06D2E323
:1051D000BE06E2B3BE0650281F4298051FD29A05AC
:1051E0000F93482492432A0282432C0208430F3C27
:1051F0000F480F5F0B4F0F5F0F5F0F5B8F43BE03B7
:1052000092522A022A0292622C022C0218533890DF
:1052100020002E2C92B298052A02042092B29A0500
:105220002C02E6270B481B530F480F5F0E4F0F5FF2
:105230000F5F0F5E8F4BBE030B480B5B0B5B0F4882
:105240000F5F0E4F0F5F0F5F0F5E9F4B3A02C00361
:105250009F4B3C02C2030F480F5F0B4F0F5F0F5F66
:105260000F5B9F420202C4039F420402C603C83F71
:1052700082430005E2E3BE06B2902000000502284A
:1052800030407869C293BB0602205E43013C4E4326
:105290005F42BA065FF34FBE0220304078691F427A
:1052A00000050F5F0B4F0F5F0F5F0F5B8F93BE0308
:1052B0007B24F240440081061F4200050F5F0B4F24
:1052C0000F5F0F5F0F5BD24FBE038406F24285066D
:1052D0001F4200050F5F0B4F0F5F0F5F0F5BD24F39
:1052E000C00386061F4200050F5F0B4F0F5F0F5F65
:1052F0000F5BD24FC10387061F4200050F5F0B4FA4
:105300000F5F0F5F0F5B1E4FC203C24E88061F4226
:1053100000050F5F0B4F0F5F0F5F0F5B1E4FC0034A
:105320001F4FC2038F104E4F0F43C24E89061F42BC
:1053300000050F5F0B4F0F5F0F5F0F5BD24FC40372
:105340008A061F4200050F5F0B4F0F5F0F5F0F5B59
:10535000D24FC5038B061F4200050F5F0B4F0F5F37
:105360000F5F0F5B1E4FC603C24E8C061F42000527
:105370000F5F0B4F0F5F0F5F0F5B1E4FC4031F4F7D
:10538000C6038F104E4F0F43C24E8D06F2402900C8
:1053900082061F4200050F5F0B4F0F5F0F5F0F5B11
:1053A0008F43BE03D243BB06925300053040786959
:1053B000F292B90602243040BC63C293C106752044
:1053C00092B3A201582C824328025A42C0064A4A8C
:1053D000D253C006B2B000012E021628B2B00001AE
:1053E0002E021A28B290C900440116285E421C0001
:1053F0007EF080005F42C0064F4F3FF01F005EDF2F
:10540000227BC24E1D00083C5F42C0064F4F3FF05A
:105410001F00D24F027B2100A29342010A2C0A5A9C
:105420000A5A1E4240010F438A5EB6028A6FB802D2
:10543000093C0A5A0A5A1E4242010F438A8EB6029A
:105440008A7FB8023A4014000F4A0A4F3A530F932A
:10545000FB23F2902000C0060928C243C0069253E5
:105460003603C293C2060224D243C106C293C106C8
:10547000022092D3A00192B38201022C3040A8589E
:10548000824382011F4290013F50983A824F92011D
:1054900092539401B2900A009401022C3040A85813
:1054A00082439401D243C206FF3DC293C00624202A
:1054B000924340038243420382433C0382433E03C0
:1054C000A2C3A001B2B000042E020928C2431D00ED
:1054D000F24024008100F240A5008200063CF24028
:1054E00014008100F24095008200A2D3A00192D363
:1054F000A001B250100036035F42C0064F4F0F5F4D
:105500000F5F1C4FB6021D4FB8021E4236030F4EEE
:105510003FE30F5F0F7FB012D279824C3002824D91
:1055200032025F42C0064F4F0F5F0F5F9F42300253
:10553000B6029F423202B8025F42C0064F4F0F5F71
:105540000F5F9F5FB602B6029F6FB802B8029F5FFF
:10555000B602B6029F6FB802B8029F5FB602B602EB
:105560009F6FB802B8029F5FB602B6029F6FB80283
:10557000B802B29300FC53241E4200FC0F4E3FE3DE
:105580000F5F0F7F828E3002827F3202829332025F
:1055900022380320929330021E281E420AFC0F4339
:1055A0001F923202043812201E9230020F2C1C422D
:1055B00030021D4232021E4202FC1F4204FCB012A5
:1055C000967A824C3002824D3202493C824330024C
:1055D00082433202443C1E420AFC0F431C4230020A
:1055E0001D4232023CE33DE31C530D630F9D033823
:1055F00011200E9C0F2C1C4230021D4232021E4212
:1056000006FC1F4208FCB012967A824C3002824D92
:105610003202253C8243300282433202203C1E4249
:1056200030021F4232023C40543E1D43021232C23D
:105630000343824E3001824C3801824E3401924243
:105640003A01300292423C013A01824D3801824FC8
:105650003401824C380192423A0132023241924284
:10566000320218028293980536245F42C0064F4FDB
:105670000F5F1F4F36021F5298051F9218020B38FA
:105680005F42C0064F4F0F5F1F4F36021F829805C3
:10569000829F180220343C4000010B4C5C42C00643
:1056A0006E42B0127E794E4C0C4BB012127A82DCF4
:1056B0004C045F42C0064F4F0F5F9F4218023602F4
:1056C0005C42C0066E42B0127E794C4C1C9296052C
:1056D000023492D35A045F42C0064F4F0F5F9F427D
:1056E000180276025F42C0064F4F0F5FBF90CEFF99
:1056F00076020D341E4244031F4246031EF240034D
:105700001FF2420382DE3C0382DF3E030E3C5F4217
:10571000C0064F4F0F5FBF90C4097602063492D285
:1057200040033C0392D242033E03925240034003A3
:10573000926242034203D253C006F2902000C00698
:10574000B32892B3A201FD2F82934E041420B2908D
:10575000060020020A389292340244010C2CD243F3
:10576000C30682434C0430404E3A1F4244013F502E
:1057700038FF824F340292F29C053C0392F29E0560
:105780003E031E423C031F423E031EE244031FE24F
:105790004603824E3002824F3202B290060020024F
:1057A0003738C293C30634201F4230021FD2320260
:1057B0000F932E240A430B3C0C12C14A00003C41BB
:1057C000B012AC3712113202121030021A533A9052
:1057D0002000182C92B33002F52B1C423C031D42D2
:1057E0003E030E12C14A00003E41B0124A7A5CB339
:1057F000E3270C12C14A00003C417C508000B012EB
:10580000AC37E03F92423C03440392423E034603DE
:10581000C243C30682433603C243C106C243C20623
:10582000C243C006B2B000012E021628B2B0000179
:105830002E021A28B290C900440116285E421C00AC
:105840007EF080005F42C0064F4F3FF01F005EDFDA
:10585000227BC24E1D00083C5F42C0064F4F3FF006
:105860001F00D24F027B2100A2C3A001B2B00004EE
:105870002E020428F240A4008100033CF240940070
:105880008100A2D3A00192D3A001824382011F42D2
:1058900090013F50983A824F920182439401829343
:1058A00052040224B253520482934E044B25829335
:1058B000520448211F4256040F830B241F83732474
:1058C0001F838E241F83C1241F83D7241F83E624B4
:1058D000393DF2C0100029001F422E023FF00005A2
:1058E0003F9000051F20B2901000500405289243FD
:1058F0005804A2425604263DB2925004092C3C4062
:1059000080005E425004B0123C7AC24C3100463CEA
:105910001C435E4250047E50F800B012127AC24C12
:1059200021003C3CB29014005004052892435804D6
:10593000A2425604073DB2925004092C3C4080001C
:105940005E425004B0123C7AC24C3100273CB29205
:1059500050040420F2D080001D00203C1F4250045F
:105960003F8009003F920A2C1C435E4250047E5047
:10597000F700B012127AC24C2100103C1F425004B2
:105980003F8011003F900300092C1C435E425004ED
:105990007E50EF00B012127AC24C2900A24352048A
:1059A00092435604CF3C8293A4050A249292A40504
:1059B0004401062CB24003005804A2425604C23CE3
:1059C0008293A6050A2492924401A605062CB240B1
:1059D00003005804A2425604B53CA2435604B23C0C
:1059E000A2B24E04AF2CC293BB0602205E43013C20
:1059F0004E435F42BA065FF34FBEA424F24042001A
:105A00008106F24003008406F24005008506D2427A
:105A1000500486061E4244018E103EF0FF00C24E26
:105A200087061E424401C24E8806C2438906C2430D
:105A30008A06F2404A008206D243BB06B2404600C4
:105A40005204B240030056047D3CA2425604A2B365
:105A50004E040F288293A2050924F2D010002900D9
:105A60009242A2055204A24256046C3CA24358043E
:105A7000693CB24003005804653CF2C010002900A4
:105A8000C2433100F2C080001D00C2432100F2F089
:105A9000F8002900B24005005604543CA2B24E045E
:105AA000512CC293BB0602205E43013C4E435F4231
:105AB000BA065FF34FBE4624F24042008106D2434D
:105AC0008406F2428506D24250048606D242580429
:105AD0008706829358040C241E4244018E103EF027
:105AE000FF00C24E88061E424401C24E89061C3C7D
:105AF000924270011802D24202028806D242030288
:105B000089061E420402C24E8A061E4202021F423B
:105B100004028F104E4F0F43C24E8B06D242180222
:105B20008C06D24219028D06F2404B008206D24307
:105B3000BB068243560482434E0482435804B2405B
:105B4000FF005004C293BE060524C243BE06B24005
:105B500001FF4C0492921002040221280420929228
:105B60000E0202021C2892939A0519381E429A05C9
:105B70000F4E3FE30F5F0F7F1E5202021F620402AF
:105B8000824E0E02824F10021F429C051FD29E05BC
:105B90000F930524B2D030004C04A2D25A04929242
:105BA0000C0204021B28042092920A020202162808
:105BB0009293940513381E4294050F4E3FE30F5FF6
:105BC0000F7F1E5202021F620402824E0A02824F9F
:105BD0000C02B2D040004C04A2D35A04B290070089
:105BE00020023E399292440134023A2DC293BB0600
:105BF00002205E43013C4E435F42BA065FF34FBE54
:105C00002F251F4248043FF01F001F924A046724BB
:105C100092534A04B2F01F004A041A4248043AF070
:105C2000E0FF1A524A04829A4804022C3A50E0FFDC
:105C3000F240440081061F424A040F5F0F5F0F5F6E
:105C4000D24F48038406F24285061F424A040F5F82
:105C50000F5F0F5FD24F4A0386061F424A040F5F51
:105C60000F5F0F5FD24F4B0387061F424A040F5F3F
:105C70000F5F0F5F1E4F4C03C24E88061F424A043F
:105C80000F5F0F5F0F5F1E4F4A031F4F4C038F10B4
:105C90004E4F0F43C24E89061F424A040F5F0F5FEB
:105CA0000F5FD24F4E038A061F424A040F5F0F5FF9
:105CB0000F5FD24F4F038B06C24A8C068A103AF010
:105CC000FF00C24A8D06F240880082061F429C05F2
:105CD0001FD29E050F93C424D243BB06C13CB2B071
:105CE00010004C042A28F24044008106C243840676
:105CF000F24006008506D24244038606D24245039E
:105D000087061E424603C24E88061E4244031F42B7
:105D100046038F104E4F0F43C24E8906D2424804AD
:105D20008A06D24249048B06F24028008206D243FA
:105D3000BB06B2E010004C04933CB2B040004C04EF
:105D400055281A424C043AF00F0092534C040A931F
:105D50001D20F240480081065E4296057E504000BC
:105D6000C24E8406E2428506D24202028606D24232
:105D700003028706D24204028806D242050289063F
:105D8000F2406A008206D243BB066A3C3A531A923A
:105D90009605292CF24048008106F24068008206F0
:105DA0004A5A4A5AC24A84063E425D4284064D4DD2
:105DB0000D5D3D5076025C4284064C4C0C5C3C50C0
:105DC0003602B0126A7A3E425D4284064D4D0D5D48
:105DD0003D5076023C408606B0126A7AF242850651
:105DE000D243BB063D3CB2F030FF4C04B2B000FFE2
:105DF0004C0436243A4000010843023C0A5A185326
:105E0000189296052D2C82BA4C04F827F2404800CF
:105E1000810648584858C24884063E425D4284067E
:105E20004D4D0D5D3D5076025C4284064C4C0C5C41
:105E30003C503602B0126A7A3E425D4284064D4DB5
:105E40000D5D3D5076023C408606B0126A7AF24201
:105E50008506F2406900820682EA4C04D243BB0602
:105E600092B366014928C293BF062D24C293BC0693
:105E70000724B012842B92538A0592532402233CA8
:105E8000C293BB062024D242B8068306E293BB0627
:105E90000E20F2428206C2438106F2438406C243C8
:105EA0008506F240C8008106C243BB060A3CC29385
:105EB00081060538C243BA06D2428106BC06D2C367
:105EC000BB06B0121E2B92536206925366061F4207
:105ED00070013F500A003FF0FF03824F760192C3EA
:105EE0006601B290B90B66060228B0127235829331
:105EF000A8050220B0126A2CB29005005E060224AA
:105F000030405463A2935A060234304046638243C1
:105F10002602824366065F42C5064F4F1F92A805C0
:105F20000224304046635E42C4064E4E3EF04F00AF
:105F30007E8040000E245E830C246E831A245E83D0
:105F400018247E8005000E245E8359245E83572426
:105F5000FA3DC243C4062C43B012E634B2400002FC
:105F60005A04F13DF2400B00C4062C43B012E63453
:105F7000EA3DF2902D00C6062A20F2900600C806DF
:105F800026205842CA064848385038FF08585F4211
:105F9000CC064F4F1FE31FF3085FC293CC060B34B0
:105FA00082934E041F20B24005004E0482435604E3
:105FB00082485004173CB29005004E04132082988A
:105FC00050041020A2D34E04824352040B3CF290A2
:105FD0006700C6060724F2906400C6060320B2409C
:105FE00000015A045E42C4067EF04F007E904300DA
:105FF000AA21C243C4062C43B012E634A43DF242A7
:10600000C406D242A805C506D243C706D242A80597
:10601000C906C243CA06C243CB06B29000025A0464
:106020000E20F2404600C606E242C806E243CC0615
:106030003C400900B012E63482435A04BC3DB290A1
:1060400000015A041120F2406400C606F240070025
:10605000C806F2401400CC063C400900B012E634F9
:10606000B24006035A04A73DB29000045A0410201F
:10607000F2406400C606F2400A00C806F24014006E
:10608000CC063C400900B012E63482435A04933DEA
:10609000A2B24E042728A29356042420F2402D00D9
:1060A000C606F2400700C8061E42500412C30E1076
:1060B0007E50C800C24ECA065E4250045EE35EF3E4
:1060C0007E508000C24ECC063C400900B012E6343F
:1060D000B24003005604B2D000806806B2403200DD
:1060E0005204693DA2B24E042328B2900500560422
:1060F0001F20F2402D00C606F2400700C8061E42CF
:10610000500412C30E107E50C800C24ECA065E4232
:1061100050045EE35EF3C24ECC063C400900B01270
:10612000E634B24006005604B2D000406806433D53
:10613000A2B24E042628B290060056042220F24055
:106140002D00C606F2400A00C8061E42500412C3C3
:106150000E107E50C800C24ECA065E4250045EE376
:106160005EF3C24ECC063C400900B012E6348243D6
:10617000560482434E0482435804B240FF00500448
:106180001A3D1F4248043FF01F001F924A04322468
:1061900018424A04185338F01F00D243C606F24092
:1061A0008100C706F2400300C8060F480F5F0F5F6B
:1061B0000F5F5E4F48037EF07F005E535F4296059F
:1061C0004F5F4F5F4E8FC24ECA0608580858085896
:1061D000C893480302385E43013C4E43C24ECC068E
:1061E00092534A04B2F01F004A043C400900B01226
:1061F000E634E13CA2B25A043D28A2C25A043A4015
:1062000020001F4296050F5F0F5F0A8F0A9332240A
:10621000D243C6060E12C14A00003E417E508000A5
:10622000C24EC7061F425A043FF000033F900003CE
:106230000420F2401400C806023CE243C806D243E0
:10624000CA060843103C1C4244031D4246031E423A
:1062500096050E5E0E5E4E58B0124A7A5CF35CE311
:10626000C84CCC061853089AEE2B3A520C4AB0127E
:10627000E634A13CF2B003005A045224B2F0FCFF11
:106280005A041A4296050A5A0A5A0A934924F240B5
:106290000900C6060E12C14A00003E417E50800031
:1062A000C24EC7061F425A043FF000033F9000034E
:1062B0000420F2401400C806033CF2400300C80664
:1062C000F2406400CA06B24076021E02B240CC061A
:1062D0001C0208431B3C1F421E021B421C02EB4FC8
:1062E000000092531E0292531C021F421E021B42C8
:1062F0001C02EB4F000092531E0292531C021F42DD
:106300001C02CF43000092531C021853089AE32B3F
:106310000F4A0A5A0A5F3A520C4AB012E6344B3C12
:10632000F2400900C4062C43B012E6341F425A045E
:106330003FF000033F9000030420B24000045A04E1
:10634000023C82435A04B29005005E063420B0122B
:106350004635313C92935E060B20929264066206AB
:106360002A2882436206D2D32900A2435E06233C38
:10637000A2935E060E209292600662061C28B2402E
:1063800003005E06F2D020000100F2D020000300DE
:10639000123CB29003005E060E20B2B000205C06F4
:1063A0000A28D2B379000728F2C020000100D2C326
:1063B0002900B01246350A4330407869F2900A004D
:1063C000B906022430407869B29005009405022095
:1063D0003040786982933602A2251F4240020F8323
:1063E0000B241F83D3241F83F9241F8342251F837B
:1063F00069251F838B25913D1F4238020F5F924F05
:10640000D6054E021F4238020F5F924F16064C020D
:106410001F4238020F5F924F960550021F429405AB
:106420000F8307241F8310241F8323241F832D24FD
:10643000373CB290200038020228924342021A42AE
:1064400038020A5A0A5A2E3C1A42380212C30A105B
:106450000A110A110A110A5A0A5A3A50480092427D
:10646000D6054E02924216064C0292429605500202
:10647000193CB2903C0038020228924342021A4270
:1064800038023AF0FE000A5A0D3CB2902000380261
:106490000228924342021A4238020A5A0A5A023C1D
:1064A000A2434202829350020320B2400300420200
:1064B00082435202B290030094053C24F24322002E
:1064C000F2407F002A00F2431E00F2433200D24A1B
:1064D000427B2100D24A437B2900D24A447B3100CF
:1064E000D24A457B1D00D29A427B20000F205E429B
:1064F00028007EF07F005E9A437B0820D29A447B7E
:1065000030000420D29A457B1C000224A2424202A1
:106510003A903C000620F2D0100019005E421800AC
:10652000093CF2C010001900F2B010001800022857
:10653000A2424202929394052120924244024802D0
:1065400092934E020838929248024E020434B240AE
:106550000A004202133C5A42380212C34A104A4A05
:106560003AF007000A5A0A5AD24A427B2100D29ACC
:10657000427B20000324B240050042028293420283
:10658000CE2092433C0292534002C93CB29032006A
:106590003C02C53892939405172492424402480263
:1065A00082934E02072492924E0244020334B24078
:1065B0000600420282934C020724929244024C024B
:1065C0000334B2400700420282934202A820924361
:1065D0003C029253400292435202A13CB2901027D7
:1065E0003C020238B242420282933A029820B290B0
:1065F000030094051F20F2432200F2407F002A008E
:10660000F2431E00F24332001A4238020A5A0A5A72
:10661000D24A427B2100D24A437B2900D24A447BA2
:106620003100D24A457B1D003A903C000320F2D055
:106630001000190092433C02824382011F429001E4
:106640003F50DC05824F9201B29003009405032471
:10665000F2D020001900829394050424B290030024
:1066600094050320A24240025A3CB240030040027B
:10667000563CB290C8003C025238929394050A20CE
:1066800092B33802042CF2D020002900033CF2D04F
:1066900040002900A2939405082092B33802032CED
:1066A000E2D31D00023CD2D31D0092433C02824340
:1066B00082011F4290013F50DC05824F92019253AC
:1066C00040022D3C1F4250021F53829F3C0227284C
:1066D000829394050424B29003009405022092430F
:1066E0003E02929394050720F2F09F002900924306
:1066F0003C0292534002A29394051120F2F0FC0058
:106700001D0092433C0292534002093CB290C800E3
:106710003C02053892433E02023C8243400282938F
:1067200052022B24A29340022820C293BB060220CF
:106730005E43013C4E435F42BA065FF34FBE1D24E9
:10674000F24042008106F24003008406F240050058
:106750008506D24238028606D24249028706D242D4
:1067600048028806C2438906C2438A06F2404A00AC
:106770008206D243BB06824352028293360203242E
:1067800082934202032082933E026724F2C02000DB
:106790001900C2432100C2432900C2431D00C24365
:1067A0003100F2C010001900C2432200C2432A0087
:1067B000C2431E00C243320082434002824336027B
:1067C00082433C0282433E0292433A02B012122BB1
:1067D000C293BB0602205E43013C4E435F42BA06B1
:1067E0005FF34FBE3824F24042008106D243840654
:1067F000F2428506D24238028606D242420287061B
:10680000829342020724D24249028806D2424802B9
:1068100089061C3C924270011802D242020288068C
:10682000D242030289061E420402C24E8A061E425A
:1068300002021F4204028F104E4F0F43C24E8B06BE
:10684000D24218028C06D24219028D06F2404B0049
:106850008206D243BB068243420292B3A2010B2CB2
:106860009242400144029242420146029242440155
:106870004A0292D3A00192B382017E28C293BF063E
:106880002D24C293BC060724B012842B92538A0590
:1068900092532402233CC293BB062024D242B80662
:1068A0008306E293BB060E20F2428206C2438106B3
:1068B000F2438406C2438506F240C2008106C24309
:1068C000BB060A3CC29381060538C243BA06D242CF
:1068D0008106BC06D2C3BB06B0121E2B824328021F
:1068E00082438201B250DC05920182933C02022471
:1068F00092533C02829336020A20C293BE060524BC
:10690000C243BE06B2403175540292535402829380
:1069100056023220B290317554022E38C293BB0613
:1069200002205E43013C4E435F42BA065FF34FBE16
:10693000232482435402F24042008106E24384064B
:10694000E2428506D2424B028606D2424A028706BE
:10695000D24247028806D24246028906F2404900E6
:106960008206D243BB06083C82432802B290320022
:1069700070010220B0123C79B2901A00240209384A
:10698000B2903D0020020238B0127E752C42B01247
:106990008278C293280002343040443A7C402C0074
:1069A000B012B4274B4C5BB3022C3040C26EB01215
:1069B0005628C24C35075E434D437C402C00B01234
:1069C0001E28F290EB0090060820C243BC06D2437A
:1069D000BA06824324023040BE6EC2938F0632351F
:1069E00082432602F292B9060620F290C8008F0672
:1069F00002243040BE6EF2900F009206592082436E
:106A00002602D242B8068306C293BC060824B012FE
:106A1000842B92538A05925324023040BE6EC29357
:106A2000BB063124E293BB062020F2428206C24319
:106A30008106F2438406C2438506E293B906042028
:106A4000F240C40081060E3CF292B9060420F240E6
:106A5000C8008106073CF2900A00B9060320F24004
:106A6000C2008106C243BB060A3CC29381060538B8
:106A7000C243BA06D2428106BC06D2C3BB06B012DC
:106A80001E2B3040BE6EC293900602383040BE6E60
:106A9000D2C31900F24084007700F2B04000020037
:106AA000FC2B584276004848D2D319003040BE6EC5
:106AB000D2428F06AB06F242AC06D2429106AD0638
:106AC000D2429206AE06C243AF065E4292068E11D5
:106AD0003E900F00AF2C0E5E104EDC6AFA6A346BEB
:106AE0004E6B546B386C606B6A6B866BA06BA86BDB
:106AF000AE6BDA6BFA6B346C126CB24094051C020C
:106B00005E4294064E4E5F4295064F4F3FF0FF00A7
:106B10008F100E5F825E1C020843073C1F421C025E
:106B2000E84FB00692531C0218533892F72BF242EA
:106B3000AF06823C0843083C1F421C02DF48940613
:106B4000000092531C0218533892F62B753CB01279
:106B5000E475723CB0127E75B2400B5A2001FF3FC3
:106B60003C409406B012FE77673C0843073C1F4246
:106B70001E02E84FB00692531E0218533892F72BAC
:106B8000F242AF06593C5E4294064E4E5F42950675
:106B90004F4F3FF0FF008F100E5F824E1E024C3CA5
:106BA000D2429406BD06483CB0124878453CB240FB
:106BB000AA5500028243880582438A05B0127E7579
:106BC000B01200EA824C0002D2420002B006D24269
:106BD0000102B106E243AF062F3CB24094051C020D
:106BE0000843083C1F421C02DF48940600009253F1
:106BF0001C0218533892F62B1F3C5F4294064F4FED
:106C00000F5F0F5F9F4296063A029F4298063C0232
:106C1000133CB24088051C020843073C1F421C027B
:106C2000E84FB00692531C0218533892F72BF242E9
:106C3000AF06023CF243AF06F293AF064025B01216
:106C4000A22B3D3DD2938F068920D29392066A20D3
:106C5000829398060420B240D4016001033C924222
:106C6000980670019242940602029242960604022D
:106C70001C4202021D4204023E40100E0F43B0129D
:106C80009A790A4EF292B9062520184294050C4AC8
:106C90001E429405B0128279088E0E480F431E5290
:106CA00002021F620402824E0A02824F0C02184244
:106CB0009A050C4A1E429A05B0128279088E0E4837
:106CC0000F431E5202021F620402824E0E02824FC6
:106CD0001002F53CE293B906F220184294050C4AE2
:106CE0001E429405B0128279088E0E480F431E5240
:106CF00002021F620402824E0A02824F0C021842F4
:106D000096050C4A1E429605B0128279088E0E48EE
:106D10000F431E5202021F620402824E0E02824F75
:106D20001002CD3CF290030092060420F2400300D2
:106D3000BE06C53CE29292060320D243BD06BF3C8C
:106D4000F290050092060320C243BD06B83CF290C3
:106D500006009206B420E2D3BB06B13CC2938F0674
:106D60000820D2939206AB2082432602D243BF066C
:106D7000A63CE293B9061220D2933507A020F290E8
:106D800044008F069C20C293940699205F4292068D
:106D90004F4F3FF01F00824FBC03913CF292B90667
:106DA0003F20D29335071420F29044008F06102024
:106DB000C29394060D201F429C051FD29E050F937F
:106DC00007245F4292064F4F3FF01F00824F4A0454
:106DD000D29335071720F29042008F06132082933A
:106DE000A2056D24C293BD066A2482934E046720D7
:106DF00092434E04824356045F4292064F4F824FA5
:106E000050045D3CD29335075A20E2938F065720F9
:106E100092934E045420A2434E04824352044F3CAA
:106E2000F2900A00B9064B20D29335071E20F2904B
:106E300042008F061A20B290050094054024C293A8
:106E4000BD063D24829336023A2092433A02924391
:106E500036028243400282433C0282433E025F424A
:106E600092064F4F824F38022A3CF29005003507B8
:106E70002620F29042008F062220F29392061F20D5
:106E8000F2432200F2407F002A00F2431E00F24348
:106E90003200D24294062100D24295062900D24205
:106EA00096063100D24297061D00C293980604242C
:106EB000F2D010001900033CF2C010001900C243C8
:106EC00035076BB3022C3040443AB012B4294B4C16
:106ED000F2900A00B9060C20829336020924C2936C
:106EE000BD060624B2900500940502243040883F78
:106EF000F292B9060A2092934E040720C293BD066F
:106F00000424A2434E04824352046E434D437C400A
:106F10002C00B0121E28F2900A00B906022430405C
:106F2000443AB2900500940502243040443AF2906D
:106F300042009D0659205B93572058429F064848BF
:106F400008580858085808585C42A0066E43B0120A
:106F50007E794C4C085C18530A43433C0F4A0F5F40
:106F60008F9896053D200F4A12C30F100F110F1175
:106F70005C430E12C14A00003E417EF00700B01291
:106F8000127ACFBC3A022C240F4A0F5F1E4F16060E
:106F90000E5E0F4A0F5F8F4ED6050A5A0A5AD2DA92
:106FA000C27B3602D2DAC37B3702D2DAC47B380224
:106FB000D2DAC57B3902D2D2360221005E423702D4
:106FC0007EF07F00C2DE2900D2D238023100D2D258
:106FD00039021D00C29337020334F2D010001900A9
:106FE0001A533A902000BA2BF2F0E3009E06F2907A
:106FF00044009D0602243040443A7B900600022C57
:107000003040443A5A42A6064A4A5F42A7064F4FCA
:107010003FF0FF008F100A5F5F429F064F4F0F5FE8
:10702000BF40204E3E02F29020009E0628205F4284
:107030009F064F4F0F5F0F5FDF42A2065E025F4267
:107040009F064F4F0F5F0F5FDF42A3065F025F4255
:107050009F064F4F0F5F0F5FDF42A40660025F4243
:107060009F064F4F0F5F0F5FDF42A50661025F4231
:107070009F064F4F0F5F8F4A4E023040443AF290C6
:1070800080009E0602243040443A5A42A8064A4AEA
:107090005F42A9064F4F3FF0FF008F100A5F5F422B
:1070A0009F064F4F0F5F8F9A4E0202283040443A9E
:1070B0005F429F064F4F0F5F8F4A4E025A42A00613
:1070C0004A4A4A931D340B12C14A00003B4112C385
:1070D0004B104B114B114B4B3BF003005F429F0693
:1070E0004F4F0F5F0F5F0B5F5C430E12C14A0000F2
:1070F0003E417EF00700B012127ACBDC5E021C3CEF
:107100000B12C14A00003B4112C34B104B114B11F3
:107110004B4B3BF003005F429F064F4F0F5F0F5FEB
:107120000B5F5C430E12C14A00003E417EF0070037
:10713000B012127ACBCC5E023AB04000022C304042
:10714000443A1A533AB02000022C30400C3A0B1249
:10715000C14A00003B4112C34B104B114B114B4B2A
:107160003BF003005F429F064F4F0F5F0F5F0B5FC7
:107170005C430E12C14A00003E417EF00700B0128F
:10718000127ACBDC5E023040443A4F4C1FE27E065E
:107190003FF00F000F5F1E427E0612C30E100E114D
:1071A0000E110E111EEFC47A824E7E0612C34C10D1
:1071B0004C114C114C114F4C1FE27E063FF00F005A
:1071C0000F5F1E427E0612C30E100E110E110E111D
:1071D0001EEFC47A824E7E063041B2B000022E020B
:1071E0001228F2F03F001B00F2D22A00F2D0400039
:1071F0001A00F2F0CF000500F2C010000100F2C04A
:1072000020000100033CF2D0C0001A00F2D0400080
:107210001900B2B000022E020328F2D22900033C6A
:10722000F2D0800019002F433F530F93FD233041CC
:10723000F2D0400019002F433F530F93FD23B2B00B
:1072400000022E020328F2D22900033CF2D0800073
:1072500019002F433F530F93FD23F2C04000190044
:107260002F433F530F93FD23B2B000022E02032899
:10727000F2C22900033CF2C0800019002F433F53A3
:107280000F93FD233041F2C0400019002F433F53BC
:107290000F93FD23B2B000022E020328F2D2290080
:1072A000033CF2D0800019002F433F530F93FD237E
:1072B000F2D0400019002F433F530F93FD2330417C
:1072C0007D4080000F430A3CF2D0800019002E431D
:1072D0003E530E93FD2312C34D101F533F9226348D
:1072E0002E433E530E93FD23B2B000022E0203281C
:1072F000F2C22900033CF2C0800019002E433E5325
:107300000E93FD234CBD0424F2D040001900033C31
:10731000F2C0400019002E433E530E93FD23B2B03D
:1073200000022E02D12BF2D22900D13F2E433E5330
:107330000E93FD23B2B000022E020328F2C22900F0
:10734000033CF2C0800019002E433E530E93FD23F0
:10735000F2C040001A002E433E530E93FD23B2B0FC
:1073600000022E020328F2D22900033CF2D0800052
:1073700019002E433E530E93FD235F4218004F4FDA
:107380003FF040002E433E530E93FD23B2B0000267
:107390002E020328F2C22900033CF2C0800019002B
:1073A0002E433E530E93FD23F2D040001A000C4FA3
:1073B00030417D408000F2C040001A004C430F4332
:1073C0000A3CF2D0800019002E433E530E93FD2359
:1073D00012C34D101F533F9222342E433E530E933F
:1073E000FD23B2B000022E020328F2C22900033CA2
:1073F000F2C0800019002E433E530E93FD23F2B0DD
:107400004000180001284C5D2E433E530E93FD238F
:10741000B2B000022E02D52BF2D22900D53F2E4366
:107420003E530E93FD23B2B000022E020328F2C297
:107430002900033CF2C0800019002E433E530E93F6
:10744000FD23F2D040001A00F2C0400019002E4384
:107450003E530E93FD23B2B000022E020328F2D257
:107460002900033CF2D0800019002E433E530E93B6
:10747000FD232E433E530E93FD23B2B000022E0295
:107480000328F2C22900033CF2C0800019002E43F9
:107490003E530E93FD2330417D408000F2C04000FA
:1074A0001A004C430F430A3CF2D0800019002E43CF
:1074B0003E530E93FD2312C34D101F533F922234AF
:1074C0002E433E530E93FD23B2B000022E0203283A
:1074D000F2C22900033CF2C0800019002E433E5343
:1074E0000E93FD23F2B04000180001284C5D2E439E
:1074F0003E530E93FD23B2B000022E02D52BF2D2E2
:107500002900D53F2E433E530E93FD23B2B0000217
:107510002E020328F2C22900033CF2C080001900A9
:107520002E433E530E93FD23F2D040001A00F2D0BA
:10753000400019002E433E530E93FD23B2B00002CB
:107540002E020328F2D22900033CF2D08000190059
:107550002E433E530E93FD232E433E530E93FD23A5
:10756000B2B000022E020328F2C22900033CF2C08E
:10757000800019002E433E530E93FD2330410A1222
:10758000B012DA7182437E06B01230727C40A000E5
:10759000B012C0726C43B012C0724C43B012C072D1
:1075A0007C405500B012C0727C405500B0128A7108
:1075B0000A43093C5C4A3602B0128A715C4A3602C0
:1075C000B012C0721A533A905E03F42B5C427E06EE
:1075D000B012C0725C427F06B012C072B0128672E6
:1075E0003A4130410A12B012DA7182437E06B0127B
:1075F00030727C40A000B012C0724C43B012C07216
:107600004C43B012C0727C40AA00B012C0727C40E1
:10761000AA00B0128A710A43093C5C4A9405B01270
:107620008A715C4A9405B012C0721A533A90C6002F
:10763000F42B5C427E06B012C0725C427F06B01230
:10764000C072B01286723A4130410A12B012DA7139
:10765000B01230727C404300B012C072B012987405
:10766000C24CB906B0128672C243B806F293B9068C
:107670000324C293B9061120B2D000022E02B01228
:10768000DA71B01230727C404300B012C072B01296
:107690009874C24CB906B0128672C293B906023809
:1076A000D2D3B806F2B04000B906022CE2D3B80635
:1076B000F2B01000B906022CE2D2B806F2B02000F7
:1076C000B906022CF2D2B8065E42B9064E4E3EF022
:1076D0000E006E8205246E820A246E8204240A3C07
:1076E000E243B9060B3CF2400A00B906073CF242FD
:1076F000B906043C3C400300B01282788243220267
:10770000B01230727C40A000B012C0724C43B01274
:10771000C0724C43B012C072B01230727C40A100F3
:10772000B012C07282437E06B012B2734A4C0C1281
:10773000C14A00003C41B0128A710A43093CB012B0
:10774000B273CA4C94055C4A9405B0128A711A53FC
:107750003A90C600F42BB012B273B0128A71B01214
:107760009874B0128A71B012867282937E060A24CF
:10777000924322020A43033CCA4394051A533A90A7
:10778000C600FA2BB01230727C40A000B012C0725A
:107790006C43B012C0724C43B012C072B01230725F
:1077A0007C40A100B012C072B012B273B0128A71E4
:1077B0000A43093CB012B273CA4C36025C4A360224
:1077C000B0128A711A533A905E03F42BB012B2735E
:1077D000B0128A71B0129874B0128A71B0128672A7
:1077E00082937E0608240A43033CCA4336021A5396
:1077F0003A905E03FA2B925388053A413041B240E9
:10780000805A200132C20343B24051A52A010F43DE
:10781000143CB24040A52801B24000A52C011E42F4
:107820001E02EE4C00001C5392531E02B24000A5F3
:107830002801B24010A52C011F533F92EA2B32D2EF
:10784000B2400C5A20013041B240805A200132C26D
:107850000343B24051A52A01B24002A52801B2401B
:1078600000A52C011F421E02CF430000B24000A51C
:107870002801B24010A52C0132D2B2400C5A20018E
:1078800030410A120B120A4CB0123C790B43213CD6
:10789000B01214793E4060EA0F4E0E4F3E530F93E4
:1078A000FB23B0123C793E4060EA0F4E0E4F3E5330
:1078B0000F93FB233E4060EA0F4E0E4F3E530F9353
:1078C000FB233E4060EA0F4E0E4F3E530F93FB23C7
:1078D0001B530B9ADD2B3A90030019383E4060EAA7
:1078E0000F4E0E4F3E530F93FB233E4060EA0F4E68
:1078F0000E4F3E530F93FB233E4060EA0F4E0E4F58
:107900003E530F93FB23B2400B5A2001FF3F3B41F4
:107910003A413041B2B000012E020428F2D04000BA
:1079200035003041B01230727C404200B012C0725B
:107930007C40FE00B012C07230408672B2B00001CE
:107940002E020428F2C0400035003041B0123072DF
:107950007C404200B012C0727C43B012C072304012
:10796000867230406A7930406279FF3F3541344158
:1079700037413641394138413B413A4130417CF34E
:107980007EF30F4E0D4C0E431C430D5D0E6E0E9F8D
:1079900001280E8F0C6CF92B304109120A120B12C0
:1079A0000A430B43394020000C5C0D6D0A6A0B6BD7
:1079B0000A8E0B7F04281CD33953F623043C0A5E3D
:1079C0000B6F3953F1230E4A0F4B3B413A4139417A
:1079D0003041091209430F9305343EE33FE31E5340
:1079E0000F6319D30D9305343CE33DE31C530D6342
:1079F00039E3B0129A7919B304243CE33DE31C53F4
:107A00000D6329B304243EE33FE31E530F63394162
:107A100030414E9303240C5C5E83FD2330417E9005
:107A2000100004280D4C0C437E8010004E9304245B
:107A30000C5C0D6D5E83FC2330417CF34E9304247B
:107A400012C30C105E83FC2330417E901000052889
:107A50000C4D0D4309247E8010004E93052412C363
:107A60000D100C105E83FB2330410A120A4C043CBB
:107A7000EA4D00001A531D530F4E3E530F93F82347
:107A80003A4130410F4C0F5D033CCC4300001C5386
:107A90000C9FFB233041021232C20343824C30015F
:107AA000824E3801824C34011C423A0192423C0120
:107AB0003A01824F3801824D3401824E38011D4215
:107AC0003A010013000081100221833104428552E3
:107AD00006638773088489940AA58BB50CC68DD676
:107AE0000EE78FF760EA00307500204E0010270087
:107AF000881300C40900E2040071020038015568CF
:107B0000000408090A0B0C0D0E0F101112131415A6
:107B1000161720212223242526274041424344458D
:107B20004647084828681858387804442464145490
:107B300034740242226212523272014121611151A7
:107B40003171010000000200000004000000080084
:107B50000000100000002000000040000000800035
:107B60000000000100000002000000040000000806
:107B70000000001000000020000000400000000095
:107B80000000000080000000400000002000000015
:107B900010000000080000000400000002000000C7
:107BA00001000000008000000040000000200000F4
:107BB00000100000000800000004000000020000A7
:107BC00000010100000002000000040000000800A5
:107BD00000001000000020000000400000008000B5
:107BE0000000000100000002000000040000000886
:107BF0000000001000000020000000400000008095
:107C00000000000080000000400000002000000094
:107C10001000000008000000040000000200000046
:107C20000100000000800000004000000020000073
:107C30000010000000080000000400000002000026
:107C40000001FFFFFFFFFFFFFFFFFFFFFFFFFFFF41
:107C5000FFFFFFFFFFFFFFFFFFFFFFFFFFFFFFFF34
:107C6000FFFFFFFFFFFFFFFFFFFFFFFFFFFFFFFF24
:107C7000FFFFFFFFFFFFFFFFFFFFFFFFFFFFFFFF14
:107C8000FFFFFFFFFFFFFFFFFFFFFFFFFFFFFFFF04
:10EA00000C43B24000821E02073C1F421E026F4FA1
:10EA10004F4F0C5F92531E02B29000E01E02F52B86
:10EA20003F4020802C9F01243041B240805A200179
:10EA3000B24051A52A0132C203433E400020103C9F
:10EA4000B24002A52801B24000A52C018E4300006F
:10EA5000B24000A52801B24010A52C013E50000292
:10EA60003E900080ED2B3F4000803E400020133C54
:10EA7000BF9300000E24B24040A52801B24000A57B
:10EA80002C01AE4F0000B24000A52801B24010A5F5
:10EA90002C012F532E533E900080EA2B82436001BD
:10EAA0008243800132D282430002B2400B5A2001DD
:10EAB000FF3FFFFFFFFFFFFFFFFFFFFFFFFFFFFF26
:10EAC000FFFFFFFFFFFFFFFFFFFFFFFFFFFFFFFF56
:10EAD000FFFFFFFFFFFFFFFFFFFFFFFFFFFFFFFF46
:10EAE000FFFFFFFFFFFFFFFFFFFFFFFFFFFFFFFF36
:10EAF000FFFFFFFFFFFFFFFFFFFFFFFFFFFFFFFF26
:10EB0000FFFFFFFFFFFFFFFFFFFFFFFFFFFFFFFF15
:10EB1000FFFFFFFFFFFFFFFFFFFFFFFFFFFFFFFF05
:10EB2000FFFFFFFFFFFFFFFFFFFFFFFFFFFFFFFFF5
:10EB3000FFFFFFFFFFFFFFFFFFFFFFFFFFFFFFFFE5
:10EB4000FFFFFFFFFFFFFFFFFFFFFFFFFFFFFFFFD5
:10EB5000FFFFFFFFFFFFFFFFFFFFFFFFFFFFFFFFC5
:10EB6000FFFFFFFFFFFFFFFFFFFFFFFFFFFFFFFFB5
:10EB7000FFFFFFFFFFFFFFFFFFFFFFFFFFFFFFFFA5
:10EB8000FFFFFFFFFFFFFFFFFFFFFFFFFFFFFFFF95
:10EB9000FFFFFFFFFFFFFFFFFFFFFFFFFFFFFFFF85
:10EBA000FFFFFFFFFFFFFFFFFFFFFFFFFFFFFFFF75
:10EBB000FFFFFFFFFFFFFFFFFFFFFFFFFFFFFFFF65
:10EBC000FFFFFFFFFFFFFFFFFFFFFFFFFFFFFFFF55
:10EBD000FFFFFFFFFFFFFFFFFFFFFFFFFFFFFFFF45
:10EBE000FFFFFFFFFFFFFFFFFFFFFFFFFFFFFFFF35
:10EBF000FFFFFFFFFFFFFFFFFFFFFFFFFFFFFFFF25
:10FC00000000543E0100543E01000500FFFFFFFFCD
:10FC1000FFFFFFFFFFFFFFFFFFFFFFFFFFFFFFFFF4
:10FC2000FFFFFFFFFFFFFFFFFFFFFFFFFFFFFFFFE4
:10FC3000FFFFFFFFFFFFFFFFFFFFFFFFFFFFFFFFD4
:10FC4000FFFFFFFFFFFFFFFFFFFFFFFFFFFFFFFFC4
:10FC5000FFFFFFFFFFFFFFFFFFFFFFFFFFFFFFFFB4
:10FC6000FFFFFFFFFFFFFFFFFFFFFFFFFFFFFFFFA4
:10FC7000FFFFFFFFFFFFFFFFFFFFFFFFFFFFFFFF94
:10FC8000FFFFFFFFFFFFFFFFFFFFFFFFFFFFFFFF84
:10FC9000FFFFFFFFFFFFFFFFFFFFFFFFFFFFFFFF74
:10FCA000FFFFFFFFFFFFFFFFFFFFFFFFFFFFFFFF64
:10FCB000FFFFFFFFFFFFFFFFFFFFFFFFFFFFFFFF54
:10FCC000FFFFFFFFFFFFFFFFFFFFFFFFFFFFFFFF44
:10FCD000FFFFFFFFFFFFFFFFFFFFFFFFFFFFFFFF34
:10FCE000FFFFFFFFFFFFFFFFFFFFFFFFFFFFFFFF24
:10FCF000FFFFFFFFFFFFFFFFFFFFFFFFFFFFFFFF14
:10FFE000FFFFFFFFE831B432FFFFFFFF0021FFFFFB
:10FFF000FFFFFFFFFFFFFFFFFFFFFFFF00200022CB
:00000001FF
